:100000000EC028C027C026C025C024C023C022C0DF
:1000100021C020C0BEC01EC0D9C01CC01BC011243E
:100020001FBECFE5D2E0DEBFCDBF10E0A0E6B0E05E
:10003000E8E9F8E102C005900D92A437B107D9F7BD
:1000400011E0A4E7B0E001C01D92AC3CB107E1F7BC
:10005000BED020CCD5CFA895019728F0E0EAFFE0EC
:100060003197F1F7F8CF089572E07A95F1F701979B
:10007000D9F7A895089588E08DB9C59A089584E0C8
:1000800086BB86BB86BB86BB86BB86BB86BB86BB68
:1000900086BB86BB86BB86BB86BB86BB86BB86BB58
:1000A00000008FB1089594E068B378E087FB65F9AC
:1000B00068BB880F96BB96BB7A95C1F7C59A089521
:1000C000DC01FB0122E032E02E1B3F0B241B350B31
:1000D00084E0319788F086BB86BB86BB86BB86BB37
:1000E00086BB86BB86BB86BB86BB86BB86BB86BB08
:1000F00086BB86BB86BBEDCF109731F0C0DF8D93FA
:1001000041505040D9F730C08C9956958C994795FD
:10011000899956958999479560917600A0E9B0E054
:10012000A60FB11D8091A0018C3FE0F78C99A7DF4D
:10013000A6DF8C998058E82FF82F899B06C08C99F0
:100140009EDF9DDF8C998058E82FED93FD93F89406
:100150008091A0018E5F8093A00178946E5F4150E2
:100160005040E1F66093760084E086BB86BB86BB98
:1001700086BB86BB86BB86BB86BB86BB86BB86BB77
:1001800086BB86BB86BB86BB86BB2150304069F7E9
:1001900008958F938FB78F93EF93FF93E09177003C
:1001A000FF27E057FF4F8091A001825048F08093D5
:1001B000A00181918EBD81918BBDE059E0937700C4
:1001C000FF91EF918F918FBF8F9118951895A0E0B7
:1001D000B0E0ECEEF0E027CB71B614BE8EE081BD4E
:1001E00089E288BB8EE387BB789481EA91E0AAD844
:1001F000892B09F0F8C1A8951092900080E690E054
:1002000022D7892B39F480E990E061E070E04EE874
:1002100050E06DD780919000870D81BF80E991E01B
:1002200067E670E0C9D69C018430910529F0A7E605
:10023000AA2EA0E0BA2ED2C180E991E06BE670E070
:10024000BBD69C01FBE6AF2EF0E0BF2EC7C1812CD0
:10025000E2E09E2E76E0472E60E6362E51E6252E11
:1002600080E991E060E070E0E3D49C0142E0C42EBC
:1002700090E1592EB0C1A89580E991E068E770E05F
:10028000D7D49C01009709F0ABC1809181008823ED
:1002900039F380918000827171F781E890E06CE61B
:1002A00070E06CDA009739F380E990E0B5015FDA2D
:1002B00080E990E061E770E04FDA80E990E061E882
:1002C00070E04ADAA89580E990E0BDD69C010097DD
:1002D00009F07BC180E990E06CE070E04EE850E00E
:1002E00006D7892B09F07FC180918E0090918F00F5
:1002F0000C9709F078C18091980090919900A09195
:100300009A00B0919B0087559144A645B54409F0E9
:100310006AC1DD24A89580E990E068E070E04EE8CD
:1003200050E0E5D680918E0090918F00089709F0FB
:100330005AC1E0909400F0909500009196001091C1
:1003400097008091900090919100A0919200B091BF
:1003500093008C3469E4960763E5A60764E5B60765
:1003600009F4B6C08D3429E4920723E5A20724E5F9
:10037000B20778F486366DE6960764E7A60760E272
:10038000B607B9F084549944A345B04509F02BC190
:100390009FC0843661E6960764E7A60761E6B60764
:1003A00009F463C086569146A346B44709F01BC1C1
:1003B0008FC0C70181709070892B29F00894E11CCF
:1003C000F11C011D111DD801C7014097A109B109F8
:1003D00085359105A105B10508F005C180E990E0DA
:1003E000B7014EE850E083D680918E0090918F0047
:1003F000A0E0B0E08E159F05A007B10709F0F3C09B
:1004000080919000813009F0EEC0D09092008D2D47
:100410008150823008F0E7C0D1BA90919E009830A8
:1004200019F0903109F0DFC081B3892B81BB94FDB5
:10043000DD0C2091940030919500409196005091F0
:100440009700DA01C90180549F41A040B040815417
:100450009C49A040B04008F0C6C060E874E88EE156
:1004600090E0BFD9215029BD55CFDD2009F4BBC094
:1004700080E0E81684E0F80680E0080780E01807CE
:1004800008F4B1C08D2D90E001979C01442737FD01
:100490004095542FDA01C9018E219F21A023B12359
:1004A0000097A105B10509F09EC08091B701909118
:1004B000B801A091B901B091BA01282339234A2388
:1004C0005B23211531054105510509F08CC01AC087
:1004D000C70181709070892B29F00894E11CF11CF0
:1004E000011D111D8091B7019091B801A091B90132
:1004F000B091BA01E80EF91E0A1F1B1FC801B7010F
:1005000082D208CF80B7882381F447BC3CBC20BE90
:10051000CABCC3BE59BEDD24D394DEBCDBBC84E6BA
:1005200090E0A2DD90E8D916B9F71092A0011092E0
:100530007700109276008091B7019091B801917088
:10054000B401681B790B80E090E04EE850E0CFD515
:1005500080918E0090918F00A0E0B0E0E81AF90A37
:100560000A0B1B0BDD24D394A895A1E0EA16A4E0A6
:10057000FA06A0E00A07A0E01A0718F0C0E0D4E0ED
:1005800001C0E70180E090E0BE014EE850E0AFD549
:100590009C010097D1F480918E0090918F00C81734
:1005A000D90799F4DD0CB09904C0D394B1E0DB16FF
:1005B00061F0C050D44049F480E09CEFAFEFBFEF52
:1005C000E80EF91E0A1F1B1FCFCF8091A0018823C0
:1005D000E1F76EBC6BBC232B31F44DCE80E8682E66
:1005E000232B09F434CEA89513BE1ABC80B78823F8
:1005F00059F010E811501EBD1BBD84E690E034DDBB
:100600001123C1F710BE1CBC8DE481BD85B7877E68
:10061000806185BF85B7806285BF889585B78F7DEE
:1006200085BFA8958EE081BDE0CDA0E0B0E0EAE115
:10063000F3E003C96C01C0917400D0917500FC0116
:100640001182108224813581468157812130310504
:100650004105510509F45BC08E819F81A885B9854C
:10066000281739074A075B0708F051C021153105E3
:100670004105510539F48881833021F42E853F8569
:1006800048895989F6012087318742875387211588
:1006900031054105510579F18EEFE82E8FEFF82EE7
:1006A0008FEF082F8FEF182FE20EF31E041F151F78
:1006B0008E819F81A885B9850297A109B109E816A5
:1006C000F9060A071B0728F020E030E040E050E080
:1006D00016C02A8130E040E050E0C801B70168D878
:1006E0009B01AC018A899B89AC89BD89280F391F80
:1006F0004A1F5B1F04C02E853F8548895989F60132
:10070000248735874687578720E030E002C021E004
:1007100030E0C901CDB7DEB7E8E0ABC8A4E0B0E097
:10072000E3E9F3E084C84B015C01609074007090D1
:10073000750082E088169104A104B10408F4B0C0E9
:10074000F30186819781A085B18588169906AA064E
:10075000BB0608F0A5C08081823009F45DC08330FB
:1007600009F478C0813009F09BC0C4019695879543
:10077000880D991D9C013170892F992786956C01F0
:10078000EE24FF24F3014285538564857585CE01EF
:100790000196F1E02F3F3F0749F0C40ED51EE61E3B
:1007A000F71EB701A60102E010E01DC04C0D5D1D53
:1007B0006E1D7F1D2FEF31E001E010E004D7892B83
:1007C00009F06EC0F30142855385648575854F5FDE
:1007D0005F4F6F4F7F4F4C0D5D1D6E1D7F1DCE0116
:1007E000029620E030E0EFD6892B09F059C06981EC
:1007F0007A81C40181709070892B39F0A4E07695DC
:100800006795AA95E1F79B0122C09B0140E050E06B
:100810003F704070507048C077276B2D5A2D492D7E
:10082000F30182859385A485B585480F591F6A1FFA
:100830007B1F94013070220F331FCE01019602E01E
:1008400010E0C1D6892B61F589819A819C0140E035
:1008500050E02AC0B501A40127E076956795579529
:1008600047952A95D1F7F30182859385A485B585AF
:10087000480F591F6A1F7B1F94012F773070220F7A
:10088000331F220F331FCE01019604E010E09BD6E8
:10089000892B31F429813A814B815C815F7004C0DE
:1008A00021E030E040E050E0B901CA012496EEE0DA
:1008B000DAC7A0E0B0E0EEE5F4E0BDC75C01C091AE
:1008C0007400D0917500FC01C080D1800894C11CD7
:1008D000D11CC114D10409F48FC024853585468507
:1008E0005785211531054105510509F485C0C6011B
:1008F0008F709070892B09F079C02F5F3F4F4F4F59
:100900005F4F2487358746875787408551856285A5
:100910007385411551056105710539F48C819D81FF
:10092000C816D90608F462C067C08A8190E00197B2
:100930009601E4E036952795EA95E1F78223932323
:10094000892B09F053C0CB01BA01E8DE9B01AC0151
:10095000623071058105910518F421E030E04EC048
:100960008E819F81A885B985281739074A075B07BB
:1009700008F042C0F5012087318742875387C09134
:100980007400D09175000EEFE02E0FEFF02E0FEFF8
:10099000002F0FEF102FE20EF31E041F151F8E8184
:1009A0009F81A885B9850297A109B109E816F906C2
:1009B0000A071B0728F020E030E040E050E011C0BB
:1009C0002A8130E040E050E0C801B701F1D69B0138
:1009D000AC018A899B89AC89BD89280F391F4A1FC0
:1009E0005B1FF5012487358746875787F501D1823C
:1009F000C08220E030E002C023E030E0C901CDB782
:100A0000DEB7EAE034C7A0E0B0E0E8E0F5E00BC70D
:100A1000E82FC0917400D0917500209719F426E05A
:100A200030E001C1898180FD03C025E030E0FBC0DA
:100A3000EA8CFB8C0C8D1D8D4E2F592FCB01DA01CA
:100A40003C014D01E614F7040805190510F43701BF
:100A50004801EE88FF88088D198D1E8A1F8A188E1E
:100A6000198E611471048104910409F4D6C08A813D
:100A7000A82EBB24CC24DD24B9E0AA0CBB1CCC1CC2
:100A8000DD1CBA95D1F7E114F10401051105A1F1BE
:100A90001701280108942108310841085108C401B0
:100AA000B3016150704080409040A601950199D6F5
:100AB00079018A01C201B101A601950192D6E2161F
:100AC000F30604071507C0F088279927DC018A1967
:100AD0009B09AC09BD0982219321A421B5218E8BEC
:100AE0009F8BA88FB98F681A790A8A0A9B0A2AA154
:100AF0003BA14CA15DA132C02E8D3F8D48A159A1D3
:100B00002AA33BA34CA35DA329C0CA01B90106DEF9
:100B10009B01AC01623071058105910508F480C02C
:100B20008E819F81A885B985281739074A075B07F9
:100B300008F076C02AA33BA34CA35DA38E899F89AE
:100B4000A88DB98D8A0D9B1DAC1DBD1D8E8B9F8BF5
:100B5000A88FB98F6A187B088C089D08A614B70463
:100B6000C804D90490F2EE88FF88088D198DE60C30
:100B7000F71C081D191DEE8AFF8A088F198F8090B7
:100B8000740090907500AEEFAA2EAFEFBA2EAFEFC3
:100B9000CA2EAFEFDA2EA20EB31EC41ED51EF4016C
:100BA00086819781A085B1850297A109B109A81610
:100BB000B906CA06DB06A0F5228130E040E050E02D
:100BC000C601B501F5D59B01AC01F4018289938979
:100BD000A489B589280F391F4A1F5B1F21153105CC
:100BE00041055105E9F0F9E016950795F794E7946A
:100BF000FA95D1F78A8190E00197AA2797FDA095F1
:100C0000BA2FE822F9220A231B232E0D3F1D401F75
:100C1000511F2EA33FA348A759A720E030E003C0EF
:100C2000198221E030E0C901CDB7DEB7E2E117C695
:100C3000ACE2B0E0EDE1F6E0FEC57C016B01809135
:100C4000740090917500892B19F426E030E0B6C04D
:100C5000CE010196D70113969C938E93129761153E
:100C6000710541F023E030E08DE0A82EB12CAC0EF0
:100C7000BD1E28C0C701D9DC9C01A0C0F70120819E
:100C800031812F70307015E0220F331F1A95E1F774
:100C9000C50100E210E097D4892B19F021E030E083
:100CA00020C09D85992309F48DC0888D953E29F03B
:100CB0009E3219F08F7383FF20C0C701FADD9C01BB
:100CC000009779F4D7011C964D915D916D917C91BF
:100CD0001F97411551056105710581F621153105F3
:100CE00061F0F701148615861686178623303105C4
:100CF00021F02115310509F061C09601275F3F4FB2
:100D0000F70184859585A685B7850097A105B1056E
:100D100009F443C0FE013D96AE014B5E5F4F8081FA
:100D2000803251F0853009F485EED9018D939D0113
:100D30003196E417F50799F78D89803299F08EE2A4
:100D4000F90181939F01FE017596AE01485E5F4FE8
:100D50008081803239F0D9018D939D013196E4175D
:100D6000F507B1F7888DF6018087FE013D96448D29
:100D7000558D668D778DD6014D935D936D937C93E4
:100D80001397808D918D15969C938E9314978689D9
:100D9000978917969C938E931697F9011082C70135
:100DA00088DD9C018330910549F4D7011C961D9282
:100DB0001D921D921C921F9720E030E0C901AC9655
:100DC000EAE055C523E030E08CCFA0E0B0E0EAEEE9
:100DD000F6E02CC57C015B016A0103C00894C11CCC
:100DE000D11CD6018C918032C9F38F3219F408944A
:100DF000C11CD11CF7011482158216821782D601FC
:100E00008C91813230F4C70110DCEC01F5011082C5
:100E1000C2C0A0E25A2E88248394FBE06F2E712C6E
:100E20006A0C7B1CD7011296CD91DC911397FE01C1
:100E3000CE010B9601C05192E817F907E1F730E0B7
:100E4000992448E002C038E04BE0F601E90DF11DBD
:100E5000208193942132A8F12F3299F12E3211F092
:100E6000341728F0483069F52E3269F32AC0822FF2
:100E700081588F3118F08F558D31C0F4A32FB0E019
:100E8000842F90E00197A817B90784F4F601E90DC3
:100E9000F11D90819394AC0FBD1F2C93832F8F5F16
:100EA000FE01E80FF11D90833E5FCFCF822F815668
:100EB0008A3108F42052FE01E30FF11D20833F5FC9
:100EC000C4CF1B86213208F48B86C701AEDBEC0150
:100ED0000097A1F5F70144855585668577852081C2
:100EE00031812F703070E5E0220F331FEA95E1F772
:100EF000C50100E210E067D3892B19F081E090E092
:100F00001CC0D5018C91882309F44AC0F30180816B
:100F100083FD0FC0F701A281B381F501E615F70546
:100F200009F441C090818C91981719F4319611966B
:100F3000F5CFC701BEDC009769F2EC01C330D105E3
:100F400051F5D7011296ED91FC9113978385882373
:100F500001F121C0F301808184FF1BC0C90CD11CA9
:100F6000D50154968D919C915597A0E0B0E0DC019D
:100F700099278827F501228D338D40E050E0822BA0
:100F8000932BA42BB52BF70184839583A683B7837A
:100F900049CFC4E0D0E0CE01CDB7DEB7EFE062C408
:100FA000C3E0D0E0CBCFD7011296ED91FC9113971F
:100FB0008385882379F2EFCFACE2B0E0E1EEF7E091
:100FC0003EC48C01AB018091740090917500892B17
:100FD00019F426E030E033C0CE010196F801938386
:100FE00082833DE0E32EF12CEC0EFD1EC801B7011B
:100FF000ECDE9C010097F1F48D858823C1F0888D8B
:1010000084FF1BC0F70184899589A0E0B0E0DC0172
:1010100099278827228D338D40E050E0822B932B37
:10102000A42BB52BF80184839583A683B783C801CD
:10103000FCDA9C012330310511F424E030E0C901D1
:10104000AC96E6E018C4ACE3B0E0E8E2F8E0F7C341
:10105000AC0100917400109175000115110519F48F
:1010600066E070E040C0F8011182CE010196988BD5
:101070008F876DE1E62EF12CEC0EFD1ECE010D9654
:10108000B701A3DEBC01009771F58D8D882349F16E
:1010900088A584FD26C0F70184899589A0E0B0E089
:1010A000DC0199278827228D338D40E050E0822B88
:1010B000932BA42BB52BF801868F978FA0A3B1A3F8
:1010C000F701848D958DA68DB78DF801828F938F52
:1010D000A48FB58F168A178A108E118E81E08183B6
:1010E00002C063E070E0CB01EC96E6E0C4C3A0E090
:1010F000B0E0ECE7F8E099C33C016B014A01C09114
:101100007400D0917500FA0111821082209719F4B1
:1011100026E030E0CAC0898180FD03C025E030E0D0
:10112000C4C02A8D3B8D4C8D5D8D8E899F89A88D85
:10113000B98D281B390B4A0B5B0BCB01A0E0B0E04B
:10114000281739074A075B0708F469015301412C46
:10115000E2E05E2EA0C02E893F89488D598DDA01CC
:10116000C9019170A070B0700097A105B10509F098
:101170005EC0DA01C90179E0B695A7959795879584
:101180007A95D1F7FA80FA94F822C9F4211531053D
:101190004105510529F46E8D7F8D88A199A105C067
:1011A0006AA17BA18CA19DA1B9DA6230710581058C
:1011B000910508F477C06AA37BA38CA39DA300913B
:1011C0007400109175002AA13BA14CA15DA1225091
:1011D000304040405040F80186819781A085B1851C
:1011E0000297A109B109281739074A075B0708F0D8
:1011F00059C0628170E080E090E0DAD29B01AC01DE
:10120000F80182899389A489B589280F391F4A1F5B
:101210005B1F211531054105510509F443C02F0D10
:10122000311D411D511D2EA33FA348A759A72E894B
:101230003F893170C201821B930B76018C159D058D
:1012400008F47C016114710419F480E090E001C09D
:10125000C5014EA15FA168A579A58701B4D1892BED
:1012600009F5C701A0E0B0E02E893F89488D598D6E
:10127000280F391F4A1F5B1F2E8B3F8B488F598FBA
:10128000AE0CBF1CCE18DF08F401808191818E0D59
:101290009F1D91838083C114D10409F05CCF20E0AD
:1012A00030E003C0198221E030E0C901CDB7DEB7DC
:1012B000E0E1D7C2A0E0B0E0EFE5F9E0BCC2B82EB3
:1012C000A92E6A017B012EEF31E002E010E07BD114
:1012D000892B11F023E031C0CB2DDA2D8881998143
:1012E00085559A4A11F022E028C08B2D9A2DB7011E
:1012F000A60126E330E002E010E065D1892B39F445
:10130000888199818654914411F420E016C08B2D78
:101310009A2DB701A60122E530E002E010E053D19A
:10132000892B11F021E009C020E088819981865441
:10133000914409F421E081E02827822FCDB7DEB760
:10134000EAE095C2A4E2B0E0E7EAF9E070C25C012D
:101350001092750010927400009709F4E6C063D1F2
:1013600080FF03C022E030E0E8C04E010894811CF9
:10137000911CC40140E050E060E070E09BDF8130F0
:1013800021F0CC24DD24760119C0C40140E050E0F6
:1013900060E070E02EEB31E000E110E014D1892B29
:1013A00009F0C6C08D81882309F4C5C0C984DA84D8
:1013B000EB84FC84C401B701A6017CDF833009F40F
:1013C000B7C0882309F0B7C0CE010196B701A601C6
:1013D0002DE030E004E210E0F6D0892B09F0A8C03F
:1013E0008A859B85BC0180E090E0611571058105CF
:1013F000910521F4688D798D8A8D9B8D2C8130E04B
:1014000040E050E0D5D13B014C018A819B81A0E0B6
:10141000B0E0C80ED91EEA1EFB1EF501C286D386B7
:10142000E486F586898182832D813E8135832483FC
:101430008F8198857C0100E010E0E114F104010542
:10144000110521F4EC88FD880E891F898A819B8112
:10145000A0E0B0E0E81AF90A0A0B1B0BE618F7083F
:1014600008091909B4E036952795BA95E1F7C9013D
:10147000A0E0B0E0E81AF90A0A0B1B0BF501228183
:1014800030E040E050E0C801B701ABD12E5F3F4FE4
:101490004F4F5F4FF5012683378340875187273FA2
:1014A000FFE03F07F0E04F07F0E05F0710F481E056
:1014B00001C082E0275F3F4F4040504008F083E08A
:1014C000F5018083833029F488A199A1AAA1BBA149
:1014D00009C0F50182859385A485B585860D971D84
:1014E000A81DB91D86879787A08BB18BF5018481D4
:1014F0009581A4E096958795AA95E1F7A0E0B0E0E4
:101500002285338544855585820F931FA41FB51FFF
:10151000860D971DA81DB91D828B938BA48BB58B4F
:101520001182B0927500A092740020E030E005C0F6
:1015300021E030E002C027E030E0C901A496EEE0EF
:1015400092C1DF92EF92FF920F931F93D82E7A01F0
:101550008B0187FF0AC087E740E050E060E070E061
:10156000F0DF823050F58FE7D822C39A88D5C39830
:1015700086D58D2D98D5812F9927AA27BB2793D55E
:10158000C801AA27BB278FD5BB27A12F902F8F2D4E
:101590008AD58E2D88D580E4D81611F485E906C049
:1015A00088E4D81611F487E801C081E07CD51AE000
:1015B00066D587FF02C01150D9F71F910F91FF9098
:1015C000EF90DF900895A0E0B0E0E8EEFAE035C1DA
:1015D0006C0179018091CB0183FD07C039E0440F94
:1015E000551F661F771F3A95D1F781E5AADF88233B
:1015F00089F4C0E3D5E743D58F3F19F42197D9F794
:1016000009C08E3F39F4C601B701A80159D500E0E1
:1016100010E002C001E010E0C39A31D5C801CDB797
:10162000DEB7E8E026C1A4E0B0E0E8E1FBE005C1F8
:1016300022D50AE010E023D501501040E1F7C3980D
:1016400008E512E01CD501501040E1F780E440E0CD
:1016500050E060E070E075DF813009F05EC088E442
:101660004AEA51E060E070E06CDF8130B1F56E0174
:101670000894C11CD11C76018E010B5F1F4FFFD453
:10168000F70181937F01E017F107C9F78B81813062
:1016900009F043C08C818A3A09F03FC008EA11E69C
:1016A00003C001501040C9F189EE40E050E060E015
:1016B00070E447DF8823A9F73CC0E1D4F6018193A9
:1016C0006F01EE15FF05C9F7898186FD03C0E4E0CF
:1016D000FE2E24C07CE0F72E21C089EE40E050E0D1
:1016E00060E070E02EDF823028F061E4E62EFF2417
:1016F000F39404C059EEE52E42E0F42E08EA11E618
:1017000003C00150104049F08E2D40E050E060E0F1
:1017100070E017DF8823A9F716C0FF24F092CB01F1
:10172000C39AADD480E0FF2009F481E02496E8E07C
:10173000A0C08AE740E050E060E070E002DF88236C
:1017400009F4BBCFEACF80E540E052E060E070E012
:10175000F8DE882311F7E2CFFB01DC010D900020B9
:10176000E9F7119701900D920020E1F70895FB0130
:10177000DC0101900D920020E1F70895FB015191E9
:101780005523A9F0BF01DC014D9145174111E1F747
:1017900059F4CD010190002049F04D9140154111BF
:1017A000C9F3FB014111EFCF81E090E0019708956B
:1017B000FF27EE27BB27AA2760FF04C0A20FB31F95
:1017C000E41FF51F220F331F441F551F9695879561
:1017D0007795679589F70097760771F7CF01BD0177
:1017E0000895A1E21A2EAA1BBB1BFD010DC0AA1F62
:1017F000BB1FEE1FFF1FA217B307E407F50720F07A
:10180000A21BB30BE40BF50B661F771F881F991FF4
:101810001A9469F760957095809590959B01AC013D
:10182000BD01CF0108952F923F924F925F926F9228
:101830007F928F929F92AF92BF92CF92DF92EF9260
:10184000FF920F931F93CF93DF93CDB7DEB7CA1BE1
:10185000DB0B0FB6F894DEBF0FBECDBF09942A880C
:10186000398848885F846E847D848C849B84AA84B4
:10187000B984C884DF80EE80FD800C811B81AA8141
:10188000B981CE0FD11D0FB6F894DEBF0FBECDBF0C
:08189000ED010895F894FFCF6B
:101898006F736363616C0077617600002E57415661
:0418A800002F00000D
:00000001FF
